:020000040000FA
:040000008A01AC2C99
:02000800882D41
:10001000C72C5334503452344F3447342034563480
:1000200065347234203433342E3439340D340A3488
:10003000003450343E342034003450343E342034C4
:10004000003443345634203400343D3420340034FA
:10005000563461346C3475346534203400342134C2
:100060004F34003421344534073400344D346F3478
:100070006434653400344F344B3400344E346F34C0
:100080002034413463346B3400344F347634653477
:100090007234723475346E34073400348A01A1002E
:1000A0005720003A03190800F720210A4E28820041
:1000B0002B302C020319BD2AFE3E0319C12A5B30E6
:1000C0002C020318612D3C302C02031C612D0030E2
:1000D0008A003C302C0282075F2B612D5F2BF32CB2
:1000E000612D3B2B6C298A29612D612DC52B612D3A
:1000F000612D612D612D612D8629A72A8829EE2A7F
:10010000E12B612DC62B1E2B012C612D9329D02BA9
:10011000612D612DEE2B00308A003A088207BA2D3E
:10012000C22DC42DC52DC82D9B2D982DAA2DA72DD0
:10013000B82DB52DB32DB02D00308A00510882079F
:100140000B2E0D2E102E1C2E1F2E4F2E522E5F2EDC
:10015000622E6F2E722E7E2E7F2E802E812E822E6C
:10016000832E842E852E862E872EA430BC00BC0BB9
:10017000B7280800BD00BD0DBD0DB520BD0BBD28C5
:100180000800561CC1280030C828561CC528FF305E
:10019000D700D801D9000330D3001430D200561054
:1001A0000800031783128D0083168C130C1483121E
:1001B0000C0803130800031783128D0075088C00C8
:1001C00083168C130C158B1355308D00AA308D00BF
:1001D0008C14000000008B17031383120D1EEE28F1
:1001E0000D12831603170C110313831208000C1E43
:1001F000F7280718FE28871AFB2800290619FE2869
:1002000099000800071286108C1E0229981C0B29E1
:10021000181218161A081A0808000D30F7200A30AC
:10022000F7200800063E831C1829313EF7200800FD
:100230002A3EF7200800A2006830F720220E0F396E
:10024000122122080F3912210800A2001E29A40041
:10025000A3012A292730A5001030A600422112212F
:100260000330A500E830A60042211221A501643028
:10027000A600422112210A30A600422112212408A0
:1002800012210800A8012608A40203184B290130F6
:10029000A302031C51292508A302031C5729A80AFD
:1002A00043292608A4070318A30A280808002608DB
:1002B000A4070318A30A2508A307280808000800B4
:1002C000A20061302202031C6A297B30220203183B
:1002D0006A29A2122208080003302D06031D832973
:1002E00083162008220424048312031D8329831605
:1002F000210623062506013A8312031D83298B015B
:1003000007308A00132F32304E200800A91608004B
:10031000A9120800E0229C210318612D01302D064E
:100320000319452AF729E0229C210318612D013089
:100330002D0603191A2ACB29831620082104031D30
:10034000A629831221304E20031408000430200215
:10035000031CB0290038031DA1292108031DA12970
:10036000831203100800C20101308316A102031C8E
:10037000A0020310A00CA10C8312C20C0310831660
:10038000A00CA10C8312C20CC20EC20CC20C8316AC
:10039000A10A831208008316220883120319D529A3
:1003A00028304E2032304E200800B3217D30831695
:1003B000A00021088312BE00C622561A08008D2212
:1003C000E422D611783042048316A00083128316EB
:1003D00023088312BE008D22E022D619F3293E3075
:1003E0004E200D2108003B304E200D2108008316C1
:1003F000220883120319FD29D02983160130A10296
:10040000031CA0028312C622561A08007C308316F1
:10041000A0048312831623088312BE006E22E022FA
:10042000D619162A3E304E200D2108003B304E20B2
:100430000D21080025304E20B3217D308316A00009
:1004400021088312BE00C622561A08008D22E4221B
:10045000D6110030C100703042048316A000831210
:100460004108BE008D22D619392AC10A031D302A3F
:10047000402A4108BE003E081B21E0220D21080051
:10048000E0223E304E200D21080025304E208316FC
:100490000130A102031CA0028312C622561A0800D2
:1004A00078308316A0048312E730BE000830C10004
:1004B000C0016E22D6195E2A03145F2A0310C00DF4
:1004C000E422BE03C10B592A4008BE008316A011C6
:1004D000201583126E22D6193B2A402AD6110830E5
:1004E000BF00561C712A1430D200831620088312D4
:1004F000D700DA00831621088312D800DA063E08F6
:10050000D900DA060430D3005610561C852AD619B5
:100510008C2ABF0B732A08000800D6110830BF00D0
:10052000561C902A1430D200831620088312D7005C
:10053000D9003E08D800D9060330D3005610561C07
:100540009F2AD619A62ABF0B922A080008002D0858
:100550000319B32A831621088312AA0083162008E0
:100560008312A90008004D30F7203D30F7202908FC
:100570001B212A0825210D2108002A16C622D61281
:100580000800861160102A12B80108000E30BF0062
:10059000DE018615601456125613D612D611C120EC
:1005A000BF0BCF2A4F08DE0018305E020318EA2A7C
:1005B0005617D6160630BF00C120BF0BDC2A080034
:1005C000E4228611601008000A30C300C120C30B6A
:1005D000E62A08008611601056160800561CEE2AFE
:1005E0000E30D2002D08D3005730BB00A03084005D
:1005F0000008031D612D840A0008DD00840A040838
:10060000B4003B0884005D088000840A0408BB0035
:1006100034088400AD0BF82AAA19102356100800DC
:100620005308BF00D30A57308400DD010008DD06FF
:10063000840ABF0B162B5D08800008005330F7209A
:100640003D30F72044081B21450825212030F720A4
:1006500046081B21470825212030F7200608C0390D
:100660001B212030F72063081B2162082521610827
:1006700025210D2108002D08031D472B25304E2074
:100680003708A4003608A3002A210D21080083168C
:1006900021088312B700831620088312B600003A9F
:1006A000031D592BB71B592B29120230AD06031D10
:1006B0000800283036020318612D29160800291079
:1006C0003C302C06031929142D08031D752B2530E9
:1006D0004E20380827212F30F7207E3029191C3072
:1006E000A9180E3027210D21080083162008031DAC
:1006F000842B21088312B800F030A9198030291901
:10070000E030380503190800B801831232304E205A
:100710000800380803192910B5232918A12B0F3018
:10072000A9197F3029191F3038060319672BB80A19
:10073000B90B8F2B672B380803192914BD232918EF
:100740008F2BA91DAD2B023038060319B803B80B47
:10075000AA2B672BB90BA12B672B02302919043068
:100760003806031DA72BB801672BB901B90A840A03
:100770003E3000060319B62B0800B901B90A840AF5
:100780003C3000060319BE2B080008000230D120BF
:10079000A9000130D120AA000330D120DF000800D9
:1007A0005F08F5000330DB202908F5000230DB206C
:1007B0002A08F5000130DB205D30F5000030DB2039
:1007C0000800861160102A121F10831682309F00C5
:1007D000831281309F00D101DE01080001302D0617
:1007E000031D0800AA129730E40083160130210689
:1007F0000319FC2B831208008312AA16A330E4000D
:10080000080001302D06031D0A2C831621088312CF
:10081000E400080064081B210D210800840AC03090
:100820000406031403190800000860218000031463
:100830000D3A03190800031008000F2403180800DC
:10084000203000060319282C09300006031D08007B
:10085000840A1D2CAF01AE010310291B7F2C000858
:10086000423A03198E2C0008483A03197D2C0008DF
:10087000443A03195B2C03189A2C30308002031C75
:10088000902C0A3000020318AA2CAF0DAE0D2F08D1
:10089000B3002E08B2000310AF0DAE0D0310AF0D64
:1008A000AE0D0310000833070318AE0AAF07031894
:1008B000AE0A3208AE070E243B2C03189A2C3030B7
:1008C0008002031C902C0A300002031C712C113092
:1008D0008002031CAA2C063000020318AA2C0A303E
:1008E0008007800E0430B1000310800DAF0DAE0DF7
:1008F000B10B752CB00B7D2C9A2C0E245D2C5D2C2D
:1009000003189A2C30308002031C902C0230000215
:100910000318AA2C00180314AF0DAE0D0E24802C62
:10092000303080072030000603199A2C0930000669
:10093000031DAA2C0408B400A0302D072D07840045
:100940002E088000840A2F088000AD0A3408840035
:100950000310080003140800601000308600EF3018
:1009600087008316FF308500C5308600AF308700D2
:1009700083128B0198018316980119309900203059
:10098000980083129030980007308A00042F831655
:100990008030810083128101D0010630BA00D60177
:1009A0005614C6230030D1205D3A0319DD2C0C30DB
:1009B000AA00A90129156030DF00831682309F004C
:1009C000831281309F00D101DE01E101E201E301E8
:1009D0009730E400A330AA1AE4008B168B17B601F7
:1009E0000330B700B8010D2109304E20AC30AB0008
:1009F000291319302A1A1D304E2007128610F401CF
:100A0000561E062D2F304E205612F62CF41D1A2D90
:100A1000F4111B303506031D112D861160102A12AA
:100A2000F62CAA1C1A2D3508F7200D3A031D1A2D95
:100A30000A30F7207418282DF418242D561C002D88
:100A40002A1E002DAD26002D45304E200D21F62CFE
:100A5000AC3084001D240318F62C000860218000AF
:100A6000AC00840AAD01AF01AE013C302C06031985
:100A70003E2D3E302C0603193E2D4A2D00083C3AEF
:100A8000031D442D9B23F62C00083E3A031D4A2DDE
:100A90008923F62C51302C060319652D4F302C0676
:100AA000031929171D2403185D2DB0012A240318EA
:100AB0005F2D06302D02031C4A2D5820F62C61258F
:100AC000F62C32304E200D2108002A1260186A2DB3
:100AD000C622D612561C652D5730BB00D3010D30EF
:100AE00000060319852D103000060319840A00083A
:100AF000DD00D30A040AB4003B0884005D088000CE
:100B0000040ABB00340884006F2D10235610F62C05
:100B1000F000030EF1000A08F200000000000000DF
:100B20000408F30083010B110000640881008B2886
:100B30009826BA03DC2D98260630561C0830BA00D9
:100B40005618DC2D5730D4000830D500DC2D9826FF
:100B5000BA03DC2D98260C30D20B0830BA00DC2DFD
:100B60009826BA03DC2DBA03DC2D9826BA03DC2DB7
:100B7000BA01DC2D9826540884000130801F04300F
:100B8000BA00DC2D9826CA2DCA2D9826BA03DC2D72
:100B9000BA03DC2DBA0154088400800DD50BDC2D7E
:100BA000D40A0830D500D30BD92D0630BA0056141C
:100BB000DC2D0C30BA00DC2D8C1E0A2EE82D18120C
:100BC00018121A081A08AC30AB00F41418160A2EC2
:100BD0002B0884001A088000B500F415741EF22D4D
:100BE0007412052E103A0319741608300006031DFE
:100BF000FE2DAC300406031DAB030A2E0D3000069B
:100C0000031D052E071686147414AB0ABF300406A4
:100C1000031974159C28D10A892ED10A1F15892E13
:100C20001F19892E1E08C40083161E088312C500D2
:100C300089309F00D10A892ED10A1F15892E1F19CC
:100C4000892E4708CE001E08C60083161E08831290
:100C5000C70091309F00D10A4E084707CF00CF0C44
:100C60005008031D442ED61E3B2E5E08053E4F0243
:100C70000318D615892E561F892E5F084F02031CB4
:100C8000892E6430D000892ED00B892E5F084F0248
:100C9000031C892E5616561386116010892ED10A10
:100CA0001F15892E1F19892E1E08C80083161E08BD
:100CB0008312C900831299309F00D10A892ED10A6C
:100CC0001F15892E1F19892E1E08CA0083161E089B
:100CD0008312CB008312A1309F00D10A892ED10A42
:100CE0001F15892E1F19892E1E08CC0083161E0879
:100CF0008312CD00831281309F00D10AD10AD10A1C
:100D0000D10AD10AD10AD10AD10AD10AD10A0130B5
:100D1000D100E10F8F2EE20F8F2EE30A000073083F
:100D2000840072088A00710E8300F00E700E0900B4
:100D30000608CF3986000000000000000000000017
:100D4000000000000000601C0800E018AA2EE0145B
:100D500086160800E010061608000E30D200023099
:100D6000D3003708D700A919D42E38081F39291DF8
:100D70000F39D800291DC02E0310D80C031858169F
:100D80005817291CD816291AE02E5308BF00D30A79
:100D900057308400DB010008DB06840ABF0BCB2E32
:100DA0005B08800056100800D30A3F30D80038088E
:100DB000D900D9172918D9135908291AE02EC52E98
:100DC000D30A5908DA005808D9003708D80036087D
:060DD000C038D700C52E5B
:100E000007308A00022F000083120313061C132FE1
:100E10009927D427831203178C0883120313031D09
:100E2000132F8A0108284C30BB273E30BB270D30DA
:100E3000BB270A30BB27B0273A3A031D1B2FA3015B
:100E4000A0271F39A2000310A20CA027A000A027F2
:100E5000A1000310A00CA10CA027013A0319882FB0
:100E60002508003A031D7F2FE030200703187F2F4D
:100E7000273084002208A400A0278000840AA0272D
:100E80008000840AA40B3C2FA0272308031D962F63
:100E9000071686149927D427831203178C08831208
:100EA0000313031D592F99273F308E00FF308C000C
:100EB000C827273084002208A40007302002031C22
:100EC000672F031D7F2F0030210203187F2F20087A
:100ED000831203178F008312031321088312031751
:100EE0008D0000088C00840A00088E00840AC82740
:100EF00083120313A10F7D2FA00AA40B5D2F0716E9
:100F000086142E30BB270D30BB270A30BB271B2F82
:100F1000B027B0275330BB270D30BB270A30BB2783
:100F200099278E018C01C8278A0108284630BB27E3
:100F3000982F8312031707308F0003308D000800AD
:100F4000B027BF3E031C073E0A3EA500A50EB027F2
:100F5000BF3E031C073E0A3EA5042508A307080060
:100F600083120313071286108C1EB42F1A0807165B
:100F70008614BB270800831203130718C22F871A91
:100F8000BF2FC42F0619C22F0C1EC42F99000800B2
:100F90008316031784308C0055308D00AA308D00E5
:100FA0008C140000000008001F308F058316031703
:0C0FB00080308C000C14000000000800D1
:02400E00323F3F
:08420000000000000000600056
:00000001FF
